:1000000000308A0004280000FF238316900000308F
:100010008A001F2826308400000803191E2801309A
:10002000D800D701D70B1228D80B11284A30D70097
:10003000D70B182800000000800B0F280034840123
:100040001F30830507309F001030A0000C30D70010
:1000500007308101813084000008F03907388000C2
:1000600064000008F039570480006400FA30A600EC
:100070000A206400FA30A6000A206400FA30A600C4
:100080000A206400FA30A6000A2064002014A0149C
:100090002015A01120120130A50020088700FF3094
:1000A0008316850020308700640083122015200805
:1000B0008700A3012308F93C031C6028A30A5A28DF
:1000C000201120088700A3012308F93C031C6A289B
:1000D000A30A6428250B7728A01420142008870081
:1000E0000030871A0130003A031D7728A501A508C2
:1000F000031D80282010A010A015201620088700BE
:0601000083165428630081
:02400E00AD31D2
:00000001FF
